:100000000C9435000C945D000C945D000C945D0024
:100010000C945D000C945D000C945D000C945D00EC
:100020000C945D000C945D000C945D000C945D00DC
:100030000C945D000C945D000C945D000C945D00CC
:100040000C945D000C945D000C945D000C945D00BC
:100050000C945D000C945D000C945D000C945D00AC
:100060000C945D000C945D00B90111241FBECFEF0C
:10007000D4E0DEBFCDBF11E0A0E0B1E0E4EFF3E0FB
:1000800002C005900D92A637B107D9F723E0A6E785
:10009000B1E001C01D92AB30B207E1F710E0CAE653
:1000A000D0E004C02297FE010E94F401C836D107B7
:1000B000C9F70E94B4000C94F8010C94000020E0F1
:1000C00030E080E061E070E04A9BFECFEFE9FFE0C6
:1000D0003197F1F700C000004A9B08C0AB01022E27
:1000E00002C0440F551F0A94E2F7842B4A99FECFB1
:1000F0002F5F3F4F2830310539F70895CF934A9944
:1001000024C08FE19EE40197F1F700C000004A99F6
:100110001FC04A9BFECF4A99FECF0E945F0081110B
:100120001AC00E945F008F3EC9F40E945F00C82F72
:100130000E945F002C2F30E0A901480F511D4F3F56
:10014000510571F02FEF30E00BC02FEF30E008C009
:100150002FEF30E005C02FEF30E002C02FEF30E08E
:10016000822F932FCF910895789482E390E027E532
:1001700031E0E0ECF0E0A6ECB0E07DE06AE011C038
:10018000408145FFFDCF5C9359915111F9CF4081DA
:1001900045FFFDCF7C93408145FFFDCF6C930197D8
:1001A00019F0E90157E4ECCF299AC0ECD0E006EC55
:1001B00010E00F2EF0E6EF2EF1E0FF2EF02D0F2EC7
:1001C000FDE0CF2EF02D0F2EFAE0DF2EF02D4A9914
:1001D000FECF289A0E947E00B82EAC015527888158
:1001E00085FFFDCF80E3D8018C9360E070E0CB0108
:1001F0009695879596958795969587959C01220F5C
:10020000331F880F991F880F991F880F991F820F1E
:10021000931F681B790B605D888185FFFDCFF80116
:1002200060839A013695279536952795ABE7B4E11B
:100230000E94E60196958795805D988195FFFDCF98
:10024000D8018C939A01ADECBCEC0E94E601FC0154
:10025000F695E795F695E795F695E7959F010E9447
:10026000E6019695879596958795969587959C0135
:10027000220F331F880F991F880F991F880F991F0E
:10028000820F931FE81BF90BE05D888185FFFDCF8E
:10029000D801EC939A01ADECBCEC0E94E601969576
:1002A000879596958795969587959C01220F331F84
:1002B000880F991F880F991F880F991F820F931F0E
:1002C000481B590B405D888185FFFDCFF8014083B5
:1002D000F70190E2888185FFFDCFD8019C93919131
:1002E0009111F8CF888185FFFDCFF801C082888108
:1002F00085FFFDCFD801DC92BFEFBB1209C0EFE74D
:10030000F4E82EE1E150F0402040E1F700C00000A9
:1003100028985DCFCF93DF93789481E88093C400D1
:100320001092C00088E08093C10086E08093C200F4
:10033000ACE6B1E095E5E0ECF0E0C6ECD0E0808121
:1003400085FFFDCF98839D919111F9CFE0ECF0E00E
:10035000808185FFFDCF8DE08093C600E0ECF0E06A
:10036000808185FFFDCF8AE08093C600DF91CF9129
:1003700008958AE093E00E948A01559A539A239A3D
:1003800081E284BD81E085BD16BC1092B60091EA81
:100390009093B0008093B1001092B20010926E0062
:1003A0001092700018BC1092B4001092B300209A02
:1003B000219A2898299856985E9857985F9810BE69
:1003C00010927B0083E080937F000895A29FB0018C
:1003D000B39FC001A39F01D0B29F700D811D112456
:1003E000911D0895EE0FFF1F0590F491E02D0994E3
:0403F000F894FFCFAF
:1003F4000A0D0A0D52656365697665643A200A0D33
:100404004F464620094F4E00696E74204952736965
:10041400676E616C5B5D203D207B002F2F204F4673
:10042400462C204F4E2028696E2031302773206FD0
:1004340066206D6963726F7365636F6E6473290000
:100444002C20007D3B0047656C6164656E210020B3
:1004540050726573736564210D0A005561727420CE
:06046400646F6E652100CB
:00000001FF
